:020000020000FC
:0200000016C028
:02002800099439
:10002C00099408E00EBF0FEF0DBF0FEF0AB9009354
:10003C00D90002B908B900E001B907B90FE003BB58
:10004C00279A2F9807E804B900E50CBD01E00DBD17
:10005C00E0E0F2E001E000937E0000E000937C0021
:10006C0007EE00937A0090E080E0D0E0C0E874E006
:10007C0060E00CE70093DD0014E34BD01CE062D091
:10008C0012E060D014E345D01EE05CD013E05AD0EF
:10009C0014E33FD010E056D017E154D014E339D01C
:1000AC0012E050D017E14ED014E333D014E04AD014
:1000BC0019E748D014E32DD016E044D019E742D00C
:1000CC0014E327D01AE03ED010E03CD014E321D04A
:1000DC0018E038D012E136D014E31BD010E132D046
:1000EC0010EA30D014E315D012E12CD011E02AD054
:1000FC0017E014BD10E016BD10E817BD13E0109307
:10010C006E00789400000000000000000000000069
:10011C00F9CF00E006BD00E207BD01E004BD749814
:10012C0075986C986D98A99BFECF00E006BDA99AB6
:10013C006D9AA99BFECF6C9A00E006BDA99AA99B6B
:10014C00FECFA99A28E000E006BD00E207BD01E061
:10015C0004BD110F10F06D9A01C06D98A99BFECFD4
:10016C006C9800E006BDA99AA99BFECF6C9A00E0A2
:10017C0006BDA99AA99BFECF00E006BDA99A2A95B7
:10018C0041F76D98A9994DCF6599FCCFA99BFECFEE
:10019C006C9800E006BDA99AA99BFECF6C9A00E072
:1001AC0006BDA99AA99BFECF00E006BDA99A00E85E
:1001BC0007BDA99936CF659BFCCF00E004BD08951F
:10040000E9E28827992760E022271FEF0196621F03
:10041000613061F08BB99093DA0064BB11B917B900
:1004200022B928B9A29A21B927B9F0CF80E090E08B
:100430006627C0E0DDEF44245524A0E0B6E0A09399
:100440000002B0930102CC2401E0D02E0CE0802EFB
:100450001895289A5EBC289801968A179B0710F079
:10046000882799271DB517FFFDCF7EB44EBC7C0DA4
:10047000CD1DD61FCA17DB0710F0CC27DD271DB511
:1004800017FFFDCF6EB45EBC8BB99093DA0064BBEE
:100490001FEF11B917B962B878B8A29A61B967B9F4
:1004A0001DB517FFFDCF1EB54EBC8E010BB91093C5
:1004B000DA0051E0050F161F60B026B10A171B07BE
:1004C00010F0002711273DB537FFFDCF3EB50BB922
:1004D0001093DA000000000070B036B1472F40954D
:1004E00024032001649E410C561E102D3703400C3E
:1004F000511C779E100D411C561E8E013D017694B5
:1005000067940615170518F4060D171D02C0061985
:1005100017090BB91093DA00050F161F60B026B14A
:100520000A171B0710F0002711270BB91093DA00E8
:100530000000000070B036B124031001649E210C4D
:10054000361E102D3703200C311C779E100D211CF8
:10055000361E8E01272F081B190B30F400951095BD
:100560002095250F061F161F3D01769467940615EA
:10057000170540F00A1B1B0B009510952095250FC1
:10058000061F161F3D0177FC07C0660C771C220F63
:10059000001F111F77FEF9CF220F001F111F601AD5
:1005A000710AA301920131032001209F3001300321
:1005B000560A700C411C561E129F700C411C561E90
:1005C00091013503400C511C249F600C711C461E88
:1005D000561E3403560A700C411C561E529F700C56
:1005E000411C561EEA9429F510E4E12E1091DB001F
:1005F00010FF02C0E8941DC0E6F0689411FF0CC023
:1006000001E08016B0F08A948F01FCE4E82DEE0F33
:10061000C590D490F8010DC008E1801648F4839489
:100620008F01FCE4E82DEE0FC590D490F80101C0D5
:10063000802E0091000210910102A017B10718F05E
:1006400019F0129701C0129610917A0014FF38C069
:100650000091780010917900A00EB11E961E17EF40
:1006600010937A00FA9461F59694B794A7949694AF
:10067000B794A79400E012E0A016B10608F4580160
:1006800000910002109101020A191B0918F401954A
:10069000161F11950034160730F00EEFA022A0921D
:1006A0000002B0920102AA24BB2499240091DB002D
:1006B00008770695069512E0010F0F13EE27F02F2D
:0206C00018958B
:10080000E9E28827992760E022271FEF0196621FFF
:10081000643061F08BB99093DA0064BB11B917B9F9
:1008200022B928B9A29A21B927B9F0CF80E090E087
:1008300060E0C0E0DEEF77E00024A1E0BB27CC243D
:1008400001E0D02E55272224332444245524E89453
:100850001895289A3EBC28981DB517FFFDCF7EB489
:100860002EBC74BBCBB9D093DA002196721F737083
:10087000746020B036B01DB517FFFDCF6EB45EBCFE
:100880008BB99093DA0064BB1FEF11B917B962B846
:1008900078B8A29A21B927B91DB517FFFDCF9EB42C
:1008A0004EBC74BBCBB9D093DA000196621F637063
:1008B00040B056B01DB517FFFDCF8EB48BB99093E5
:1008C000DA0064BB1FEF11B917B982B898B8A29AC1
:1008D00021B927B90196621F6370EC01762F4EF49F
:1008E00004E0C00ED21E521FC014DA065B0748F0A7
:1008F000E89402E0C01AD20A520B19F404E0C02EA8
:100900006894CC19DD09750B7370746010917A00CE
:1009100014FF32C00091780010917900300FA11EB1
:10092000B21E17EF10937A00EA9431F5B694A794AB
:10093000379511E0A116B20610F4A12E33278501D8
:10094000432F40190A0B1B0B18F440950095109586
:1009500040380207120718F0D5013C7F032EAA2465
:10096000BB2433270091DB0008770695069512E03B
:0A097000010F0F13EE27F02F18956A
:100C0000E3E28827992760E022271FEF0196621F01
:100C1000643061F08BB99093DA0064BB11B917B9F5
:100C200022B928B9A29A21B927B9F0CF81E090E082
:100C300060E0C1E0DFEF77E033272224332444244F
:100C40005524E8941895289A3EBC28981EF00196E1
:100C5000621F63701DB517FFFDCF7EB42EBC1DB59E
:100C600017FFFDCF6EB45EBC66F08BB99093DA00CF
:100C700064BB1FEF11B917B962B878B8A29A21B94D
:100C800027B91DB517FFFDCF9EB44EBC1EF00196CF
:100C9000621F63701DB517FFFDCF8EB4E6F18BB9EF
:100CA0009093DA0064BB1FEF11B917B982B898B8F6
:100CB000A29A21B927B91301240134FD0CC037FDD4
:100CC00019C000E019E3772012F460947094601664
:100CD000710638F49FC012E0C11AD20A09F4332712
:100CE00099C030E88C01562F00501840520B5370B9
:100CF000680190C036FD0FC08601452F1A0F4B1FAB
:100D0000437080179107640709F084C0EC01762FC7
:100D1000306468940CC035FD0AC07370CC15DD05D5
:100D2000750729F430620FEFC02ED02EE894239778
:100D3000720B7370746074BBCBB9D093DA002196D8
:100D4000721F7370746020B036B074BBCBB9D0938F
:100D5000DA000000000040B056B035FF5BC000E88C
:100D600010E0C01AD10A11F008F007C013012401E5
:100D700000E01FE0680130614DC060920002709297
:100D800001028101A60115031001049F3001140323
:100D9000320A700C211C321E509F700C211C321E16
:100DA0000091000210910102409550951503200C0E
:100DB000311C049F600C711C221E321E1403320A67
:100DC000700C211C321E509F700C211C321E82019F
:100DD000A60115032001049F30011403520A700C70
:100DE000411C521E509F700C411C521E84014095A4
:100DF00050951503400C511C049F600C711C421E41
:100E0000521E1403520A700C411C521E509F700C4B
:100E1000411C521E10917A0014FF31C000917800DD
:100E200010917900E00EA11EB21E17EF10937A0008
:100E3000FA9429F512E0A116B20610F4A12E07C00B
:100E400000E01CEEA016B10610F0A02EB12E850118
:100E50000A1B1B0B18F40195121F11950230120783
:100E600008F0D501AA24BB24EE240091DB0008770A
:100E70000695069512E0010F0F13EE27F02F189537
:10100000E1E28827992760E022271FEF0196621FFF
:10101000613061F08BB99093DA0064BB11B917B9F4
:1010200022B928B9A29A21B927B9F0CF80E090E07F
:1010300060E0C0E0DDEF44245524A0E0B6E06D019F
:101040001895289A5EBC289801968A179B0710F07D
:10105000882799271DB517FFFDCF7EB44EBC219779
:1010600010F4ED0121971DB517FFFDCF6EB45EBCE6
:101070008BB99093DA0064BB1FEF11B917B962B84E
:1010800078B8A29A61B967B91DB517FFFDCF1EB533
:101090004EBCCBB9D093DA000000000040B056B08F
:1010A0001DB517FFFDCF1EB58E013D0176946794E7
:1010B0000615170518F4060D171D02C006191709A5
:1010C0000BB91093DA000000000020B036B08E019A
:1010D000081B190B18F40195161F11953D01769404
:1010E00067940615170528F00A1B1B0B0195161FA0
:1010F00011953D0177FC06C0660C771C000F111F8F
:1011000077FEFACF000F111F601A710AA301920136
:1011100031032001209F30013003560A700C411C1E
:10112000561E129F700C411C561E91013503400C37
:10113000511C249F600C711C461E561E3403560A17
:10114000700C411C561E529F700C411C561EAC1553
:10115000BD0518F019F0129701C0129610917A008F
:1011600014FF32C00091780010917900A00EB11EDA
:10117000961E17EF10937A00FA9431F59694B7946F
:10118000A7949694B794A79400E012E0A016B10635
:1011900008F4580186010A191B0918F40195161F55
:1011A00011950034160718F00EEFA0226501AA244D
:1011B000BB2499240091DB0008770695069512E080
:0A11C000010F0F13EE27F02F189512
:10140000E0E28827992760E022271FEF0196621FFC
:10141000613061F08BB99093DA0064BB11B917B9F0
:1014200022B928B9A29A21B927B9F0CF80E090E07B
:10143000EE24C0E0DDEF44245524A0E0B6E018958A
:10144000289A5EBC289801968A179B0710F0882777
:1014500099271DB517FFFDCF7EB44EBC219710F420
:10146000ED0121971DB517FFFDCF6EB45EBC8BB9A2
:101470009093DA00E4BA1FEF11B917B962B878B8DF
:10148000A29AE1B8E7B81DB517FFFDCF1EB54EBC57
:10149000CBB9D093DA000000000040B056B01DB5C3
:1014A00017FFFDCF1EB58E01081B190B10F40A0F94
:1014B0001B1F56F020E034E002171307F0F5689484
:1014C00044275527405850409E012050344010F486
:1014D0002A0F3B1F2BB93093DA000000000060B0E8
:1014E00076B0820115032001049F100114035E08E9
:1014F000300C411C5E1C509F300C411C5E1C830153
:10150000BA01609570951703400C511C069F200C82
:10151000311C4E1C5E1C16035E08300C411C5E1C08
:10152000709F300C411C5E1C4058504018F4E9017B
:10153000E89403C011F4E901E894AC15BD0518F076
:1015400019F0129701C0129610917A0014FF32C060
:101550000091780010917900A00EB11E9E1C17EF2B
:1015600010937A00FA9431F59694B794A7949694D0
:10157000B794A79400E018E0A016B10608F458014B
:1015800086010A191B0918F401951E1D11950034D6
:101590001E0518F00EEFA0226501AA24BB24992491
:1015A0000091DB0008770695069512E0010F0F13F6
:0615B000EE27F02F189554
:10180000E5E28827992760E022271FEF0196621FF3
:10181000643061F08BB99093DA0064BB11B917B9E9
:1018200022B928B9A29A21B927B9F0CF88279927D8
:1018300060E0CC27DFEF77E0552701E0C02EDD2404
:1018400022243324442455241895289A3EBC2898F1
:101850000196621F63702196721F737074601DB5CC
:1018600017FFFDCF7EB42EBC74BBCBB9D093DA008A
:101870002196721F7370746020B036B01DB517FFCB
:10188000FDCF6EB45EBC8BB99093DA0064BB1FEFE2
:1018900011B917B962B878B8A29A21B927B91DB59C
:1018A00017FFFDCF9EB44EBC74BBCBB9D093DA000A
:1018B0000196621F637040B056B01DB517FFFDCF93
:1018C0008EB48BB99093DA0064BB1FEF11B917B9CE
:1018D00082B898B8A29A21B927B910917A0014FF5A
:1018E00025C00091780010917900300FA11EB21E22
:1018F00017EF10937A00EA94C9F411E03217A106A9
:10190000B20610F4A39433278501432F40190A0B24
:101910001B0B18F44095009510950130120718F034
:10192000D5013C7F032EAA24BB2433270516AC0522
:10193000BD0569F038F014E0510FC21ED21E13E04D
:10194000D12205C05250C20AD20A13E0D122FA9421
:1019500059F40091DB0008770695069512E0010F17
:101960000F1711F0EE27F02FEC01762FC51BDC09C5
:0E1970007D09737074608101120128011895C1
:101C0000E3E28827992760E022271FEF0196621FF1
:101C1000643061F08BB99093DA0064BB11B917B9E5
:101C200022B928B9A29A21B927B9F0CF88279927D4
:101C300060E0CC27DFEF77E0552701E0C02EDD2400
:101C4000222433241895289A3EBC28980196621FB6
:101C500063702196721F737074601DB517FFFDCFFE
:101C60007EB42EBC1DB517FFFDCF6EB43EBC8BB944
:101C70009093DA0064BB1FEF11B917B962B878B856
:101C8000A29A21B927B91DB517FFFDCF9EB42EBC6E
:101C900074BBCBB9D093DA000000000020B036B09E
:101CA0001DB517FFFDCF8EB410917A0014FF25C02B
:101CB0000091780010917900300FA11EB21E17EF2D
:101CC00010937A00EA94C9F411E03217A106B20623
:101CD00010F4A39433278501432F40190A0B1B0BE3
:101CE00018F44095009510950130120718F0D501B1
:101CF0003E7F032EAA24BB2433270516AC05BD0561
:101D000069F038F012E0510FC21ED21E13E0D1224A
:101D100005C05150C20AD20A13E0D122FA9459F4F4
:101D20000091DB0008770695069512E0010F0F176A
:101D300011F0EE27F02FEC01762FC51BDC097D0991
:061D400073707460189539
:10200000E5E28827992760E022271FEF0196621FEB
:10201000613061F08BB99093DA0064BB11B917B9E4
:1020200022B928B9A29A21B927B9F0CF88279927D0
:1020300060E0CC27DFEF74E0552701E0D02ECC2400
:1020400022243324442455241895289A3EBC2898E9
:10205000019621961DB517FFFDCF7EB42EBCCBB9DE
:10206000D093DA000000000020B036B021961DB5F4
:1020700017FFFDCF6EB45EBC8BB99093DA0064BBE2
:102080001FEF11B917B962B878B8A29A61B967B9E8
:102090001DB517FFFDCF9EB44EBCCBB9D093DA006F
:1020A0000000000040B056B001961DB517FFFDCFEF
:1020B0008EB48BB99093DA0064BB1FEF11B917B9D6
:1020C00082B898B8A29A61B967B910917A0014FFE2
:1020D00027C00091780010917900A00EB11E361F24
:1020E00017EF10937A00EA94D9F43695B794A79431
:1020F0003695B794A79401E0A616B00610F4AA246A
:10210000B02E85010A0B1B0B18F40195161F1195B3
:102110000034160710F0D501AC7FAA24BB24332766
:10212000AC15BD0541F020F014E0C10ED61E03C071
:1021300012E0C11AD60AFA9459F40091DB0008772C
:102140000695069512E0010F0F1711F0EE27F02FFC
:08215000EC01CC19DD09189522
:10240000289A5EBC2898019674E060E01DB517FF1D
:10241000FDCF7EB44EBC74BBEC01C654D140CBB9E9
:10242000D093DA000000000040B156B11DB517FF8F
:10243000FDCF6EB45EBC8BB99093DA0064BB1FEF26
:1024400011B917B962B878B810E0A29A11B917B9E2
:102450001DB517FFFDCF9EB44EBC25E43FE35524C8
:102460004424332422241DB517FFFDCF8EB435023A
:10247000400C511C249F200C311C461E561E340358
:10248000560A300C411C561E5203560A300C411C91
:10249000561EEC01C550D240CBB9D093DA000000F3
:1024A000000040B156B128EB3AEC3502400C511C0B
:1024B000249F200C311C461E561E3403560A300C35
:1024C000411C561E5203560A300C411C561EEC018C
:1024D000CF52D340CBB9D093DA000000000040B116
:1024E00056B123EE3FE23502400C511C249F200CD4
:1024F000311C461E561E3403560A300C411C561E13
:102500005203560A300C411C561EEC01CE5FD440DB
:10251000CBB9D093DA000000000040B156B126E5F7
:1025200030ED3502400C511C249F200C311C461EFE
:10253000561E3403560A300C411C561E5203560ACE
:10254000300C411C561EEC01C652D540CBB9D0937D
:10255000DA000000000040B156B125E433E1350255
:10256000400C511C249F200C311C461E561E340367
:10257000560A300C411C561E5203560A300C411CA0
:10258000561EEC01CC5CD640CBB9D093DA000000EB
:10259000000040B156B128E43AEE3502400C511C1F
:1025A000249F200C311C461E561E3403560A300C44
:1025B000411C561E5203560A300C411C561EEC019B
:1025C000C352DA40CBB9D093DA000000000040B12A
:1025D00056B123EE3BE13502400C511C249F200CE8
:1025E000311C461E561E3403560A300C411C561E22
:1025F0005203560A300C411C561EEC01CB5EDD41E5
:10260000CBB9D093DA000000000040B156B126E506
:1026100030EE3502400C511C249F200C311C461E0C
:10262000561E3403560A300C411C561E5203560ADD
:10263000300C411C561EEC01CB50DF42CBB9D0937D
:10264000DA000000000040B156B125E43CE035025C
:10265000400C511C249F200C311C461E561E340376
:10266000560A300C411C561E5203560A300C411CAF
:10267000561EEC01CC55D943CBB9D093DA000000FB
:10268000000040B156B128E43AE03502400C511C3C
:10269000249F200C311C461E561E3403560A300C53
:1026A000411C561E5203560A300C411C561EFA9409
:1026B00039F4F091DB00F87712E0F695F695F10F1A
:0226C00018956B
:10280000E7E0EE2400E110E06801CC271895289A53
:102810005EBC28981DB517FFFDCF9EB54EBC1DB5FB
:1028200017FFFDCF8EB57EBC1DB517FFFDCF7EB463
:102830006EBC1DB517FFFDCF6EB48F016B0D7C1DF7
:10284000AD1DBE1DFD01EE0FFF1FF370F864259155
:102850003491B1FD03C021953E1D3195AB014095EA
:10286000509535032001249F100134035E08300C7D
:10287000411C5E1C529F300C411C5E1C1196FD01D8
:10288000EE0FFF1FF370F86425913491B1FD03C082
:1028900021953E1D31951197F8013703400C511CCD
:1028A000269F200C311C4E1C5E1C36035E08300C2B
:1028B000411C5E1C729F300C411C5E1C00E8500ED7
:1028C000A2019C0135032001249F100134035E08FE
:1028D000300C411C5E1C529F300C411C5E1CC0FF22
:1028E00002C040955095930135033001249F10019B
:1028F00034037E08300C611C7E1C529F300C611C1E
:102900007E1C10917A0014FF3CC000917800109159
:102910007900800E911EAE1C17EF10937A00FA9486
:1029200081F5A69497948794A694979487948401AC
:10293000442751E0150F4E1D0B191C094D0918F4C1
:1029400000951095409500341E054E0528F0B82CD2
:10295000C92CDA2CC50EDE1C88249924AA240091E7
:10296000DB0002FF02C0E89404C05EF2689411E04C
:10297000C12708770695069512E0010F0F13EE2781
:04298000F02F189587
:102C0000E4E0EE24DEE01895289A5EBC2898019650
:102C10001DB517FFFDCF7EB44EBC1DB517FFFDCF10
:102C20006EB45EBC8BB99093DA00E4BA1FEF11B9B1
:102C300017B962B878B8A29AE1B8E7B81DB517FF1E
:102C4000FDCF1EB54EBC1DB517FFFDCF1EB58F01C4
:102C50006C0D7D1DAE1DBE1DFD01EE0FFF1FF3703F
:102C6000F86425913491B1FD03C021953E1D319545
:102C7000AB014095509535032001249F100134038A
:102C80005E08300C411C5E1C529F300C411C5E1CC7
:102C90001196FD01EE0FFF1FF370F864259134913A
:102CA000B1FD03C021953E1D31951197F801370301
:102CB000400C511C269F200C311C4E1C5E1C360300
:102CC0005E08300C411C5E1C729F300C411C5E1C67
:102CD00092015D2F35032001529F410C5E1C242C74
:102CE000C52D8C0101521340552755200AF45FEF82
:102CF000050D151F0BB91093DA000000000020B17C
:102D000036B1442D409534032001249F410C5E1CB4
:102D1000302C0F5F1F4F0BB91093DA00000000003A
:102D200020B136B140953403400C511C249F300C27
:102D3000411C5E1C3201422C5C2E409450948C014C
:102D400004541440552755200AF45FEF050D151F54
:102D50000BB91093DA000000000020B136B1442D09
:102D6000409534032001249F410C5E1C302C0F5FE2
:102D70001F4F0BB91093DA000000000020B136B1EC
:102D800040953403400C511C249F300C411C5E1CA8
:102D90007594679455944794460C571CBA94A1F4C3
:102DA00010E4B12E1091DB0010FF02C0E8940CC0BB
:102DB0005EF0689411FF04C0D15030F4DD2704C0E8
:102DC00001E0D00F08F4DFEF10917A0014FF33C058
:102DD0000091780010917900800E911EAE1C17EFC3
:102DE00010937A00FA9439F5A69497948794A69450
:102DF000979487949694879496948794840150E846
:102E0000050F1E1D0C191D0918F401951E1D1195A5
:102E100000311E0518F06401C50EDE1C88249924BB
:102E2000AA240091DB0008770695069512E0010FB1
:082E30000F13EE27F02F189597
:10300000E5E0EE24C9E0D6E01895289A5EBC289841
:1030100001961DB517FFFDCF3EB54EBC1DB517FF80
:10302000FDCF2EB55EBC8BB99093DA00E4BA1FEFEA
:1030300011B917B922B938B9A29AE1B8E7B81DB5E4
:1030400017FFFDCF1EB54EBC1DB517FFFDCF1EB53A
:103050008F016C0D7D1DAE1DBE1DFD01EE0FFF1F0E
:10306000F370F86425913491B1FD03C021953E1DA4
:103070003195AB014095509535032001249F1001F7
:1030800034035E08300C411C5E1C529F300C411C06
:103090005E1C1196FD01EE0FFF1FF370F864259181
:1030A0003491B1FD03C021953E1D31951197F80172
:1030B0003703400C511C269F200C311C4E1C5E1CFB
:1030C00036035E08300C411C5E1C729F300C411CA4
:1030D0005E1C00E8500E92015D2F359F2001529F2B
:1030E000410C5E1C8C014C2F5527440F551F440F7B
:1030F000551F041B150B089405091E090BB91093E5
:10310000DA000000000020B136B1442D3403200164
:10311000249F410C5E1C302C0F5F1F4F0BB9109386
:10312000DA000000000020B136B140953403400CB5
:10313000511C249F300C410C5E1CBA9409F510E41C
:10314000B12E1091DB00012F0625012302FD5AC08C
:1031500040E86422612A12FF13C010FF02C0E89405
:103160000FC076F0689451E067FE42C011FF05C0C1
:10317000CA95C51728F4C02F03C0C50F08F4CFEFB8
:1031800010917A0014FF33C00091780010917900FB
:10319000800E911EAE1C17EF10937A00FA9439F549
:1031A000A69497948794A6949794879496948794DA
:1031B00096948794840150E8050F1E1D0C191D0973
:1031C00018F401951E1D119500311E0518F06401BB
:1031D000C50EDE1C88249924AA240091DB00087700
:1031E0000695069512E0010F0F13EE27F02F1895A4
:1031F00011FF04C0D51B20F6DD27C2CFD50F00F686
:0E320000DFEFBECF40E864266422612AB9CF1A
:10340000E4E0EE24DDE01895289A5EBC2898019649
:103410001DB517FFFDCF3EB54EBC1DB517FFFDCF47
:103420002EB57EBC8BB99093DA00E4BA1FEF11B9C8
:1034300017B922B938B9A29AE1B8E7B81DB517FF94
:10344000FDCF1EB56EBC1DB517FFFDCF1EB58F019C
:103450006C0D7D1DAE1DBE1DFD01EE0FFF1FF37037
:10346000F86425913491B1FD03C021953E1D31953D
:10347000AB014095509535032001249F1001340382
:103480005E08300C411C5E1C529F300C411C5E1CBF
:103490001196FD01EE0FFF1FF370F8642591349132
:1034A000B1FD03C021953E1D31951197F8013703F9
:1034B000400C511C269F200C311C4E1C5E1C3603F8
:1034C0005E08300C411C5E1C729F300C411C5E1C5F
:1034D00000E8500E92015D2F359F2001529F410C54
:1034E0005E1CC52D542D8C01089405091E090BB9CD
:1034F0001093DA000000000020B136B1442D3403EF
:103500002001249F410C5E1C302C0F5F1F4F0BB914
:103510001093DA000000000020B136B1409534036A
:10352000400C511C249F300C410C5E1C3201442481
:103530005D2E451A5C0A8C01089405091E090BB919
:103540001093DA000000000020B136B1442D34039E
:103550002001249F410C5E1C302C0F5F1F4F0BB9C4
:103560001093DA000000000020B136B1409534031A
:10357000400C511C249F300C410C5E1CBA94A1F4E9
:1035800010E4B12E1091DB0010FF02C0E8940CC0D3
:103590005EF0689451E011FF04C0D51B28F4DD27CC
:1035A00003C0D50F08F4DFEF10917A0014FF33C089
:1035B0000091780010917900800E911EAE1C17EFDB
:1035C00010937A00FA9439F5A69497948794A69468
:1035D000979487949694879496948794840150E85E
:1035E000050F1E1D0C191D0918F401951E1D1195BE
:1035F00000311E0518F06401C50EDE1C88249924D4
:10360000AA240091DB0008770695069512E0010FC9
:083610000F13EE27F02F1895AF
:10380000E9E18827992766271FEF8BB99093DA00A3
:1038100064BB11B917B962B968B9A29A61B967B93D
:10382000839599F7C0E2DD2722243324882458E1C8
:103830001895289A5EBC289821968E010052160B86
:103840007DB477FEFDCF7EB44EBC0BB91093DA0089
:103850000000000000B016B01DB517FFFDCF6EB41C
:103860005EBCCBB9D093DA0064BB1FEF11B917B9B6
:1038700062B878B8A29A61B967B91DB517FFFDCFD4
:103880001EB54EBC1DB517FFFDCF1EB5260C371C4F
:1038900077FC6FEF861E66272018310817FC6FEF44
:1038A000860A3101682D65957794679465957794BC
:1038B0006794659577946794659577946794659513
:1038C0007794679466278F017C0D8D1D961FFC01F0
:1038D000EE0FFF1FF370F8642591349191FD03C042
:1038E0002195361F3195472F409534032001249FA1
:1038F000410C561E402D0196FC01EE0FFF1FF37088
:10390000F8642591349191FD03C02195361F3195BE
:10391000F80101973703400C511C279F400D411CB3
:10392000561E8301112312F400951095000F111FEC
:1039300020910002309101020217130710F0980144
:1039400005C02051360B10F42227332720930002A4
:1039500030930102EA9479F410E4E12E1091DB0037
:1039600010FF02C0E89407C036F0689411FF02C04F
:103970005A9501C0539510917A0014FF35C00091FB
:10398000780010917900A00EB11E961E17EF1093CB
:103990007A00FA9449F59694B794A7949694B794BC
:1039A000A7948D010A191B0918F40195161F11958A
:1039B0000034160760F053FD07C0152F177021F073
:1039C000B694A7941A95E1F7D50153FF6D01AA2487
:1039D000BB2499240091DB0008770695069512E038
:1039E000010F0F13EE27F02F53FF16C0152F17707E
:1039F00021F0759467941A95E1F777203AF06A0EF2
:103A00007B1E48F41FEF612E712E05C06A0E7B1ECF
:103A100010F066247724630154FD03C05594479445
:103A20001895820113032001209F30011203560ACA
:103A3000700C411C561E309F700C411C561E189570
:103C0000ECE108E033E08827992722271FEF8BB9E2
:103C10009093DA0024BB11B917B922B928B9A29A36
:103C200021B927B9839599F7802FCC27DD27AA24BE
:103C3000BB24CC24DD241895289A5EBC28980196D4
:103C400021961DB517FFFDCF7EB44EBC1DB517FFE5
:103C5000FDCF6EB49EBC77FE02C060947094660C7B
:103C6000771C00E8700E1DB517FFFDCF1EB58EBC8A
:103C70008BB99093DA0024BB1FEF11B917B962B862
:103C800078B8A29A21B927B91DB517FFFDCF1EB587
:103C9000CBB9D093DA000000000040B056B0A60CBB
:103CA000B71C77FC2FEFC21ED21E2227A418B5081E
:103CB00057FC2FEFC20AD20A22274A2C5B2C1C2D5C
:103CC000332331F0032F1595579447940A95D9F76C
:103CD00042018C0111500BB91093DA0024BB4FEF55
:103CE00041B947B942B858B8A29A21B927B9061BB9
:103CF000170B0BB91093DA000000000040B056B06B
:103D0000EA94E1F410E4E12E1091DB0010FF02C010
:103D1000E89414C09EF0689411FF04C0363070F42B
:103D2000339503C0313050F03A95EC0101E0332374
:103D300021F0132F000F1A95E9F765CFA617B707E3
:103D400041F020F012E0610F721F03C011E0611B0F
:103D5000720B10917A0014FF2CC000917800109122
:103D60007900000E111E221E17EF10937A00FA94AC
:103D700001F52694179407942694179407948001CC
:103D80000A1B1B0B18F40195121F11950034120722
:103D900010F0D001AE7F0024112422240091DB001A
:103DA00008770695069512E0010F0F1711F0EE2720
:043DB000F02F189543
:10400000E1E1EE248827992761E001E0CC24D02E5D
:104010009924AA24BB244427CC27DD277727E894BA
:104020001895289A5EBC28981DB517FFFDCF3EB4A1
:104030004EBC1DB517FFFDCF2EB45EBC1DB517FFDE
:10404000FDCF1EB54EBC1DB517FFFDCF1EB50091AF
:10405000DB0002FD1AC02EF0689488279927662796
:104060003327210130FDCCC08BB99093DA0064BBBB
:104070001FEF11B917B922B838B8A29AE1B8E7B85A
:1040800001966E1D62FD31E0BBC05EF4CC27DD27DA
:104090007727E89414E1803091076E0510F480E0F2
:1040A000912F5C0DCD1DDE1D7E1D746074BBCBB9E0
:1040B000D093DA000000000040B056B08E01272FE8
:1040C00031E0030F1E1D2E1D246024BB0BB910937D
:1040D000DA000000000020B036B08201252F2095C4
:1040E00012032001029F410C5E1C302D810115033B
:1040F000400C511C059F300D411C5E1C40FD1EC034
:104100008C013327262F7370351B0C0B1D0B270BCF
:1041100034E0D39E3001C39E610C7E1C0016610604
:10412000720608F46DC0AA27BB27A0930002B093C3
:10413000010250930202A054BE0941E00091000226
:1041400010910102209102022C0D0D1D1E1D0093E5
:104150000002109301022093020234E034BB0BB939
:104160001093DA000000000020B036B031E0030FF9
:104170001E1D0BB91093DA000000000000B116B14B
:1041800012033001029F610C7E1C302D20958101AD
:104190001203600C711C029F300D611C7E1C820199
:1041A0009D0113032001029F100112035E08300CD1
:1041B000411C5E1C309F300C411C5E1C83019D0124
:1041C000209530951303400C511C029F200C311C8C
:1041D0004E1C5E1C12035E08300C411C5E1C309F9E
:1041E000300C411C5E1CA054BE0911F008F008C040
:1041F000C0910002D091010250910202772744271A
:1042000010917A0014FF2DC0009178001091790070
:10421000900EA11EBE1C17EF10937A00FA94C1F401
:10422000B694A794979410E4A10EBE1C8501292D85
:1042300028190C091D0918F42095009510952038AF
:104240000E051E0510F06501892C9924AA24BB24B3
:104250000091DB000877069506950E5F0F13EE2799
:04426000F02F18958E
:104800000000C90092015B022403ED03B6047F059A
:1048100048061107D907A2086A09330AFB0AC40B24
:104820008C0C540D1C0EE30EAB0F73103A110112D9
:10483000C8128F1355141C15E215A8166E173318DD
:10484000F918BE19821A471B0B1CCF1C931D571E4B
:104850001A1FDD1F9F2061212322E522A623672442
:104860002825E825A82667272628E528A329612AE0
:104870001F2BDC2B992C552D112ECC2E872F413040
:10488000FB30B5316E322733DF3396344D35043685
:10489000BA366F372438D9388C39403AF23AA53BCA
:1048A000563C073DB83D683E173FC53F7340214128
:1048B000CE417A422543D0437A442445CD457546BE
:1048C0001C47C34769480F49B449584AFB4A9D4BA6
:1048D0003F4CE04C814D204EBF4E5D4FFB4F9750FB
:1048E0003351CE51685202539B533254C9546055D0
:1048F000F5558A561D57B0574258D3586459F35945
:10490000825A105B9C5B285CB35C3E5DC75D4F5E6A
:10491000D75E5D5FE35F6860EB606E61F06171625E
:10492000F1627063EE636C64E8646365DD6556662E
:10493000CF664667BC673268A66819698B69FD69EE
:104940006D6ADC6A4A6BB76B236C8E6CF86C616DB8
:10495000C96D306E966EFB6E5E6FC16F2270837094
:10496000E27040719D71F9715472AE7207735F739A
:10497000B5730A745F74B27404755575A575F375D3
:1049800041768D76D87622776B77B377FA773F7852
:104990008478C77809794A798979C879057A417A1A
:1049A0007C7AB67AEE7A267B5C7B917BC57BF87B42
:1049B000297C597C887CB67CE37C0E7D397D627DC8
:1049C000897DB07DD57DFA7D1D7E3E7E5F7E7E7EBB
:1049D0009C7EB97ED57EEF7E097F217F377F4D7F1C
:1049E000617F747F867F977FA67FB47FC17FCD7FF5
:1049F000D87FE17FE97FF07FF57FF97FFD7FFE7F44
:104A0000FF7FFE7FFD7FF97FF57FF07FE97FE17F0C
:104A1000D87FCD7FC17FB47FA67F977F867F747F4D
:104A2000617F4D7F377F217F097FEF7ED57EB97E05
:104A30009C7E7E7E5F7E3E7E1D7EFA7DD57DB07D36
:104A4000897D627D397D0E7DE37CB67C887C597CD6
:104A5000297CF87BC57B917B5C7B267BEE7AB67AE2
:104A60007C7A417A057AC87989794A790979C7784F
:104A700084783F78FA77B3776B772277D8768D761C
:104A80004176F375A57555750475B2745F740A7433
:104A9000B5735E730773AE725472F9719D71407194
:104AA000E27083702270C16F5E6FFA6E966E306E28
:104AB000C96D616DF86C8E6C236CB76B4A6BDC6AE8
:104AC0006D6AFD698B691969A6683168BC674667BC
:104AD000CF665666DD656365E8646C64EE6370639B
:104AE000F1627162F0616E61EB606860E35F5D5F6F
:104AF000D75E4F5EC75D3E5DB35C285C9C5B0F5B21
:104B0000825AF3596459D3584258B0571D578956A1
:104B1000F5556055C95432549A5302536852CE51D8
:104B200033519750FB4F5D4FBF4E204E814DE04CAF
:104B30003F4C9D4BFB4A574AB3490F496948C3470D
:104B40001C477546CD4524457A44D04325437A42D7
:104B5000CE4121417340C53F173F673EB83D073DF9
:104B6000563CA53BF23A403A8C39D83824386F3756
:104B7000BA3604364D359634DE3326336E32B531CF
:104B8000FB304130872FCC2E112E552D992CDC2B4C
:104B90001F2B612AA329E52826286727A826E825B0
:104BA00028256724A623E522232261219F20DD1FDB
:104BB0001A1F561E931DCF1C0B1C471B821ABD19B2
:104BC000F81833186E17A816E2151C1555148F1314
:104BD000C81201123A117210AB0FE30E1C0E540DE5
:104BE0008C0CC30BFB0A330A6A09A208D907100709
:104BF00048067F05B604ED0324035B029201C90059
:104C00008000880090009800A100AB00B500C000B3
:104C1000CB00D700E400F20000010F011F013001BA
:104C2000430156016A0180019601AF01C801E30109
:024C3000000280
:00000001FF
